:020000040000FA
:0200000059297C
:080008001A29A00081018316F2
:100010000313C03081050800A0008101831603137B
:10002000C030810501308104831203130B110B1DB5
:100030001728A00B16280800A80005100830A000FB
:100040002D2028180514281C0510A80C2D20A00B05
:10005000212805142D202D2008001D30A100332853
:100060000830A1003328A10B33280800A90140293A
:10007000A200E1308605220D1E3986040800861391
:10008000422886170613A3002308230E38204F208A
:10009000230838204F20E130860586130800013000
:1000A0000C208616861201300C2008002608A700B6
:1000B00025126430A100672041200A30A10067208A
:1000C00041200130A1002516672041200800A00131
:1000D00021082702031C7128A00A2108A70225165F
:1000E000692830302007251E20300800B101B201F8
:1000F0000630B300080083160313981C7D28831272
:1001000003139900080087303F20290841208D30D3
:100110003F202908A600562009301C2074301C20DE
:1001200072301C2061301C206E301C2073301C206B
:100130006D301C2069301C2074301C2074301C2051
:1001400065301C2064301C2020301C2029081C2015
:1001500029087B2020301C2074301C206F301C208C
:1001600020301C206C301C2069301C206E301C207C
:100170006B301C2020301C2032301C200D301C2005
:100180000A301C2025100B1608002A08AC00DA20C3
:10019000251DD3282B08AC00DA202511981CD32864
:1001A000181218111816A510831603138C16831233
:1001B00003130800C7303F202C084120CD303F20DA
:1001C0002C08A600562009307B2074307B2072302A
:1001D0007B2061307B206E307B2073307B206D3044
:1001E0007B2069307B2074307B2074307B2065302D
:1001F0007B2064307B2020307B202C087B202C0847
:100200001C2020307B2074307B206F307B202030FE
:100210007B206C307B2069307B206E307B206B3004
:100220007B2020307B2031307B200D307B200A303A
:100230007B2008008B138B1B1A29AD00030EAE0028
:1002400083010A08AF008A0183130408B0008B18E9
:100250002C298C1A432950290B12302006183628D5
:100260000830A0002D200618A917061CA913200B82
:10027000A90CA00B32292D20061C36282514412953
:100280000B168B1050291A08AA008C1E4A291A082E
:10029000AB002515A514831603138C1283120313C8
:1002A000300884002F088A002E0E8300AD0E2D0E1C
:1002B00009008B0183160313013086058312031393
:1002C000861206138613E130860504300C200330B5
:1002D00038204F2001300C20083038204F200130CA
:1002E0000C20023038204F2001300C2028303F20D5
:1002F0000C303F2001303F2008300C2083160313C0
:100300000510061401138312031305148B100B162A
:100310008B178316031318151930990083120313D2
:100320009817831603138C169816831203130B1752
:100330001816F8308B058C018D018B17A5015C30E8
:10034000A40002308A0024085C3C4822A3001C2040
:1003500023087B20A40BA129443041207530412083
:10036000613041206C30412020304120523041200A
:10037000533041203230412033304120323041204F
:1003800020304120523041206530412063304120EF
:100390006530412070304120C0303F207430412012
:1003A000693041206F3041206E30412020304120A3
:1003B0006F3041206E3041202030412050304120AC
:1003C00049304120433041203130412036304120F6
:1003D0004630412037304120373041201A30052047
:1003E0000730132001303F20523041205830412047
:1003F00031304120203041204330412068304120BD
:1004000089303F2056304120613041206C304120FE
:10041000C0303F20523041205830412032304120FE
:10042000203041204330412068304120C9303F20F6
:1004300056304120613041206C3041201B30A400F7
:1004400002308A0024081B3CA522A3001C2023089C
:100450007B20A40B202A76202518762025188320BF
:10046000A5187620A518C520B10B2C2AB20B2C2A72
:10047000B30B2C2A40301C200D301C200A301C20CD
:1004800040307B200D307B200A307B2076202C2AC8
:1004900082070D340A344434753461346C342034AA
:1004A0005234533432343334323420345234653499
:1004B000633465347034743469346F346E340D349D
:1004C0000A343D343D343D343D343D343D343D34D7
:1004D0003D343D343D343D343D343D343D343D3494
:1004E0003D343D343D343D343D340D340A344D34D7
:1004F0006934633472346F3463346834693470340B
:10050000203450344934433431343634463437346B
:100510003734203463346F346E346E34653463346E
:10052000743465346434203461346E34643420347B
:100530007334743461346E3464342D3462347934F9
:100540002E342E342E340D340A348207723465343E
:10055000613464347934203466346F347234203436
:100560007434723461346E3473346D34693473347A
:10057000733469346F346E342E342E342E340D348B
:020580000A343B
:02400E00F23F7F
:00000001FF
